:020000001529C0
:100008002C08A0002D08A1000130A200A301640063
:100018003620031C2328A20B0B28FF30A307031844
:100028000B28A007031CA107031C1029FA30A20003
:100038000030A3000B286400362003181F288820EE
:10004800A8010830A300892036200318A80AAB1E8F
:10005800A801A20CA30B2728AB1AA213892003140A
:10006800220808003A08840038088417800484139A
:1000780000052B1B3806FF3E0800A40029080314BE
:10008800031910290B21031C0800A0002518831749
:1000980024088400200880008313A40AA9034228A6
:1000A8000408A6003A0884008030B7050830A70085
:1000B80003100318B70A6E20A60CA70B5D280000D2
:1000C800AB1A370C6E20132103146E202F08A300DF
:1000D8002E08A7288413AB1F7D28000838042B1F7F
:1000E80038068000841700083804031C380680008E
:1000F800892800083804031C38062B1B38068000A2
:10010800841738098005892837172B081F39003EBE
:10011800A1002A080E3E0318A10A371FB428371376
:10012800A0000230C620B428A40029080319102909
:100138002518831724088400000883130B21A40AB8
:10014800A9039928A301A200FF30A207031CA30753
:10015800031C10290330A100E630B420A828A1010F
:10016800FC3EA000A109031CBF28FF300000A00727
:100178000318BA28A0076400A10FB92808000310C3
:10018800A10CA00CFF3E0318C32820081029A101C8
:10019800A301A2000230DA28A101A301A2000130C4
:1001A800DA28A101A301A2000430DA28A800230854
:1001B8002102031DE128220820020430031801301F
:1001C800031902302805031DFF3010290038031DCC
:1001D800FF300405031DFF3010290404031DFF3000
:1001E80010291030A800A101A001A70CA60C031C1F
:1001F80003292208A00723080318230FA107A10C2D
:10020800A00CA50CA40CA80BF9282408102984001C
:1002180031088A00300882008313031383126400B4
:100228000800831607309F00880107108710071100
:1002380087128910091106108610061186150616F0
:1002480086168312BC01BD01D001C6018801CB010D
:10025800CD01CE01C901CF01880107108710071110
:1002680089100915D101C8018716C8308A01A6204E
:1002780087120A308A01A62087160230A300583058
:100288008A01A7208A110A12882E07150A308A01C6
:10029800B320071108000710891009150130CB0099
:1002A800640003304B028A110A1203187D293E307C
:1002B8008800C03088008A014921403088008A01BE
:1002C8004921B83088008A0149213F3088008A01D5
:1002D800492183108918831409198914091D891063
:1002E80083180915831C0911CB0A8A110A12031DE8
:1002F800542989100915080007103E3088008A0122
:100308004921891009150130CB00640003304B02E4
:100318008A110A120318CB29B830CD006400C03006
:100328004D028A110A120318BB2907108A014921B4
:10033800403088008A0149214D0888008A014921F6
:1003480007140130CE00640041304E028A110A12AF
:100358000318B62988018A014921CE0A8A110A128E
:10036800031DA729CD0A8A110A12031D9229831099
:100378008918831409198914091D89108318091506
:10038800831C0911CB0A8A110A12031D89298914B1
:1003980009110710B83088008A014921C030880047
:1003A8008A014921403088008A01492189100915AC
:1003B800B83088008A014921C03088008A01492163
:1003C800403088008A0149213F3088008A0149214C
:1003D80007148910091508000714DF304607B20012
:1003E800FF300318013EB3003208A6003308A70007
:1003F8000530A200A3018A01F520BE002508BF0030
:1004080004303E07C0003F080318013EC1003E0803
:10041800BC003F08BD003C08A0003D08A100410801
:10042800A30040088A01D2208A110A12031D412A1A
:100438008A110A1294226400513046028A110A1263
:10044800031C342AF0303C02C2000030031C013E79
:100458003D02C3008A150A12F2218A110A12372AAC
:100468008A150A1283208A014921C90ABC0A03197C
:10047800BD0A8A110A12031D0F2A8A110A128C2238
:1004880008000714D0304607B200FF300318013EB9
:10049800B3003208A6003308A7000330A200A30166
:1004A8008A01F520B2002508B30000303207BE00EB
:1004B80033080318013EBF0002303E07C0003F0862
:1004C8000318013EC1003E08BC003F08BD003C08BF
:1004D800A0003D08A1004108A30040088A01D220DD
:1004E8008A110A12031D882A8A110A1294228A1173
:1004F8000A1287278A014921C90ABC0A0319BD0AB9
:100508008A110A12031D6B2A8A110A128C2208000A
:100518008A110A12942288018A014921C90A08000D
:1005280064004908403C8A110A12031DA32A891451
:1005380009110710403088008A0149210714640016
:100548004908803C8A110A12031DB42A891009152A
:10055800CF0AC9010710403088008A0149210714D1
:1005680064004F08083C8A110A12031DC52ACF01EE
:1005780064005208013C8A110A12031DC52A07307B
:10058800CF000710B8304F0788008A0149210714A7
:10059800080064003F3049028A110A120318DB2A56
:1005A800891009154908C8008A110A12E02A891415
:1005B800091140304902C8000710B8304F078800B9
:1005C8008A0149214030480788008A0149210714D7
:1005D80008000830C900CF018A01CD22CB01640090
:1005E80014304B028A110A120318402B4B08133C93
:1005F8008A110A12031C1F2B8A110A120723C6002C
:100608008A110A121F2B03308A004B0882074734CD
:1006180072346134703468346934633420344C344F
:100628004334443420345434653472346D3469347A
:100638006E3461346C3464004608203C8A110A1216
:10064800031D392B0130CD00640004304D028A119E
:100658000A120318362B8A018C22CD0A8A110A1233
:10066800031D282B8A110A123B2B8A01F021CB0A81
:100678008A110A12031DF32A0130CD0064000530E7
:100688004D028A110A1203187A2BC9014D08CF00AE
:100698008A01CD22CB01640040304B028A110A1234
:1006A80003185F2B143088008A014921CB0A8A116C
:1006B8000A12031D4F2B4030C9008A01CD22CB01FD
:1006C800640080304B028A110A120318742B14300C
:1006D80088008A014921CB0A8A110A12031D642B5A
:1006E8000330CD078A110A12031C422BC9010530B9
:1006F800CF008A01CD22CB0164001A304B028A1147
:100708000A120318D32B4B08193C8A110A12031C2E
:10071800B22B8A110A129423C6008A110A12B22B2C
:1007280003308A004B088207533445344E3444342E
:10073800203443344F344D344D3441344E344434F2
:1007480053342034563449344134203454344534F5
:1007580052344D3449344E3441344C3464004608E4
:10076800203C8A110A12031DCC2B0130CD006400F5
:1007780004304D028A110A120318C92B8A018C22EF
:10078800CD0A8A110A12031DBB2B8A110A12CE2B1D
:100798008A014522CB0A8A110A12031D802BC9013E
:1007A8000630CF008A01CD22CB01640040304B02D5
:1007B8008A110A120318E92B3C3088008A01492162
:1007C800CB0A8A110A12031DD92B4030C9008A01AD
:1007D800CD22CB01640080304B028A110A12031823
:1007E800FE2B3C3088008A014921CB0A8A110A1263
:1007F800031DEE2BC9010230CF008A01CD22CB01A7
:1008080064000A304B028A110A120318472C4B085D
:10081800093C8A110A12031C262C8A110A12182470
:10082800C6008A110A12262C04308A004B08820757
:1008380050346F3472347434423420345034693450
:100848006E34733464004608203C8A110A12031D72
:10085800402C0130CD00640004304D028A110A1288
:1008680003183D2C8A018C22CD0A8A110A12031D15
:100878002F2C8A110A12422C8A01F021CB0A8A11E4
:100888000A12031D042C4030C9000230CF008A012F
:10089800CD22CB0164000B304B028A110A120318D7
:1008A800922C4B080A3C8A110A12031C712C8A11DB
:1008B8000A126224C6008A110A12712C04308A00B6
:1008C8004B08820750346F34723474344334203404
:1008D8005334743461347434653464004608203CFD
:1008E8008A110A12031D8B2C0130CD0064000430DC
:1008F8004D028A110A120318882C8A018C22CD0A0B
:100908008A110A12031D7A2C8A110A128D2C8A0167
:10091800F021CB0A8A110A12031D4E2C08008914F3
:1009280009110130CB00640003304B028A110A120E
:100938000318C82C0710BF3088008A0149214030AD
:1009480088008A0149210714CD01640041304D0215
:100958008A110A120318B82C88018A014921CD0A84
:100968008A110A12031DA92C8310891883140919E6
:100978008914091D891083180915831C0911CB0ACC
:100988008A110A12031D972C89100915C90107300D
:10099800CF0008004408A00042308A01CB20B200F2
:1009A8004408A00062308A01CB20B40032088400D9
:1009B80034088A01F120B400B50064003408350415
:1009C8008A110A120319682D30304502CA006400E2
:1009D8004A08003C8A110A12031D142D01308606AC
:1009E8008316061083124F08D3004908D400033039
:1009F800CF00C9018A01CD2264008A110A12061C9F
:100A08000A2D3130C6008A110A120C2D3030C6006A
:100A18008A01F0215308CF005408C9008A01CD2269
:100A280064004A08013C8A110A12031D3E2D023057
:100A380086068316861083124F08D3004908D4000F
:100A48000330CF000830C9008A01CD2264008A1122
:100A58000A12861C342D3130C6008A110A12362D2E
:100A68003030C6008A01F0215308CF005408C9006D
:100A78008A01CD2264004A08023C8A110A12031D29
:100A8800682D043086068316061183124F08D3009A
:100A98004908D4000330CF001230C9008A01CD22A2
:100AA80064008A110A12061D5E2D3130C6008A11B3
:100AB8000A12602D3030C6008A01F0215308CF0099
:100AC8005408C9008A01CD224408C60008004F080E
:100AD800D3004908D4004608D5000330CF00C90127
:100AE8008A01CD2264008A110A12061C802D313039
:100AF800C6008A110A12822D3030C6008A01F02100
:100B08000830C9008A01CD2264008A110A12861CA5
:100B1800922D3130C6008A110A12942D3030C60049
:100B28008A01F0211230C9008A01CD2264008A119D
:100B38000A12061DA42D3130C6008A110A12A62DEC
:100B48003030C6008A01F0211C30C9008A01CD224C
:100B580064008A110A12861DB62D3130C6008A112A
:100B68000A12B82D3030C6008A01F0212630C9009B
:100B78008A01CD2264008A110A12061EC82D31305E
:100B8800C6008A110A12CA2D3030C6008A01F02127
:100B98003030C9008A01CD2264008A110A12861EEB
:100BA800DA2D3130C6008A110A12DC2D3030C60029
:100BB8008A01F0215308CF005408C9005508C6001F
:100BC8008A01CD2208004F08D3004908D4004608FE
:100BD800D5000330CF004030C9008A01CD2264001F
:100BE8008A110A12071CFD2D3130C6008A110A121B
:100BF800FF2D3030C6008A01F0214830C9008A0133
:100C0800CD2264008A110A12871C0F2E3130C600CB
:100C18008A110A12112E3030C6008A01F021503094
:100C2800C9008A01CD2264008A110A12071D212EEB
:100C38003130C6008A110A12232E3030C6008A01CC
:100C4800F0215830C9008A01CD2264008A110A12A5
:100C5800871D332E3130C6008A110A12352E3030E6
:100C6800C6008A01F0216030C9008A01CD226400E3
:100C78008A110A12071E452E3130C6008A110A123F
:100C8800472E3030C6008A01F0216830C9008A0139
:100C9800CD2264008A110A12871E572E3130C600F1
:100CA8008A110A12592E3030C6008A01F02170309C
:100CB800C9008A01CD2264008A110A12071F692E11
:100CC8003130C6008A110A126B2E3030C6008A01F4
:100CD800F0217830C9008A01CD2264008A110A12F5
:100CE800871F7B2E3130C6008A110A127D2E3030C4
:100CF800C6008A01F0215308CF005408C9005508DE
:100D0800C6008A01CD2208008A014F218A0180216C
:100D18008A01ED228A016B25C9010730CF008A01BB
:100D2800CD22891009150710403088008A01492111
:100D3800BF3088008A01492107140130D2000730EA
:100D4800BA004030B8002030AA00AB01AE01AF01B4
:100D580052308A01552045308A01552041308A0198
:100D6800552044308A01552059308A0155203A309F
:100D78008A0155200A308A0155200D308A015520F4
:100D88008A016B258A01E7250730BA008030B80050
:100D98002030AA00AB01F430AC000130AD008A016C
:100DA80004208A110A12031CC42EC60064004608D7
:100DB8001B3C8A110A12031D272F0730BA00403046
:100DC800B8002030AA00AB01AE01AF0143308A0160
:100DD80055204D308A01552044308A0155203A303B
:100DE8008A0155200730BA008030B8002030AA00A8
:100DF800AB018A011F20403C8A110A12031DFD2EF7
:100E08000230A9001F30B000B101A50144308A01A9
:100E180041200730BA004030B8002030AA00AB01AA
:100E2800AE01AF010230A9005430B000B101A501F4
:100E380044308A0198200A308A0155200D308A01F1
:100E480055208A01CE244608A00008308A01CB200C
:100E5800B2005108A00005308A01D020B400320841
:100E6800840034088A01EA20B400B500640034081C
:100E780035048A110A1203195C2F0630C90206309C
:100E8800D10207104030490788008A014921071418
:100E9800CB01640006304B028A110A1203185C2F3A
:100EA80088018A014921CB0A8A110A12031D4D2F94
:100EB80064004608203C8A110A12031D652F8A0126
:100EC8008C224608A00021308A01D520B2004608AD
:100ED800A0007E308A01D020B400320834048A1180
:100EE8000A12031DC42E8A01F0210630D1076400BE
:100EF800803051028A110A12031C852F8A0193241B
:100F0800D1018A01C42E3D088A150A12031D8228C0
:100F18003C08803C8A150A12031C82288A110A128E
:100F2800992788008A150A12822808308A003C0806
:020F380000288F
:1010000082071F3411341F3401341F3400341D345F
:1010100015341734153415341F340C340A341F3486
:10102000173415341D341F3415341C341934053469
:1010300003341F3415341F34173415341F3400346F
:101040001B341B3418341834003404340A3411347B
:101050000A340A340A3411340A340434003415349E
:1010600007340E3411340D341E3405341E341F344D
:1010700015340E341F34113411341F3411340E342E
:101080001F34153411341F34053401341F34113426
:101090001D341F3404341F3411341F3411341834F8
:1010A00010341F341F340A3411341F3410341034F8
:1010B0001F3406341F341F340E341F340E341134E1
:1010C0000E341F34053402340E34093416341F3400
:1010D00005341B34163415340D3401341F340134F7
:1010E0001F3410341F340F3410340F341F340834BD
:1010F0001F341B3404341B3403341C3403341934BC
:101100001534133408003D088A150A12031DF1290D
:101110003C08EF3C8A150A12031CF1298A150A12B1
:10112000952088008A150A12F12909308A003C08A6
:02113000002994
:101200008207003400344F34003400340034073493
:1012100000340734003414347F3414347F341434ED
:1012200024342A347F342A341234233413340834D7
:101230006434623436344934553422345034003402
:1012400005340334003400341C3422344134003477
:10125000003400340034413422341C341434083453
:101260003E3408341434083408343E340834083426
:101270000034503430340034003408340834083436
:1012800008340834003460346034003400342034CE
:1012900010340834043402343E3451344934453473
:1012A0003E34003442347F344034003442346134BC
:1012B0005134493446342134413445344B3431348B
:1012C0001834143412347F34103427344534453400
:1012D000453439343C344A344934493430340134A7
:1012E00071340934053403343634493449344934CB
:1012F000363406344934493429341E340034363403
:10130000363400340034003456343634003400347B
:101310000834143422344134003414341434143472
:101320001434143400344134223414340834023474
:101330000134513409340634323449347934413477
:101340003E347E341134113411347E347F344934C8
:101350004934493436343E34413441344134223402
:101360007F344134413422341C347F34493449348D
:10137000493441347F3409340934093401343E346A
:101380004134493449347A347F34083408340834D9
:101390007F34003441347F344134003420344034CD
:1013A00041343F3401347F3408341434223441341E
:1013B0007F3440344034403440347F3402340C3481
:1013C00002347F347F340434083410347F343E34A4
:1013D0004134413441343E347F34093409340934D2
:1013E0000634080043088A150A12031DEE2A420833
:1013F000E53C8A150A12031CEE2A8A150A120422F9
:1014000088008A150A12EE2A0A308A0042088207EA
:101410003E344134513421345E347F34093419343C
:10142000293446344634493449344934313401345A
:1014300001347F34013401343F344034403440348B
:101440003F341F342034403420341F343F34403480
:10145000383440343F34633414340834143463343F
:101460000734083470340834073461345134493453
:10147000453443347F344134413400340034023441
:1014800004340834103420340034003441344134FE
:101490007F340434023401340234043440344034A0
:1014A00040344034403400340134023404340034D5
:1014B000203454345434543478347F3448344434ED
:1014C00044343834383444344434443420343834A4
:1014D0004434443448347F343834543454345434E9
:1014E000183408347E340934013402340C34523454
:1014F000523452343E347F34083404340434783463
:10150000003444347D3440340034003420344034DA
:1015100044343D347F3410342834443400340034AF
:1015200041347F34403400347C340434183404347F
:1015300078347C3408340434043478343834443413
:101540004434443438347C3414341434143408347B
:1015500008341434143418347C347C34083404349F
:101560000434083448345434543454342034043467
:101570003F344434403420343C344034403420340C
:101580007C341C342034403420341C343C3440340B
:10159000303440343C344434283410342834443417
:1015A0000C345034503450343C3444346434543467
:1015B0004C3444340834363441340034003400347C
:1015C00000347F3400340034003400344134363485
:1015D0000834003408340434083404340800630048
:0615E0008A150A12EF2A31
:02400E00753FFC
:00000001FF
